:10000000830100308A0004288301FC2CEA00EB1BEA
:1000100012286B1B1A286B088A006A08EA0A03195F
:10002000EB0A820083136B1883176A08EA0A8400BC
:100030000008080050342E345434453453346934A5
:10004000003443342E34543445345334693400344A
:10005000323430342534643425346434003450343C
:1000600041345A34413452340034533441344C34E2
:1000700049340034433455344D344134003425344C
:100080006434253464343A340034253464342534FB
:1000900064342F34003450344534523453344534AE
:1000A0002E340034433441345234533441342E34EA
:1000B00000342034533441344134543420347634C1
:1000C00065342034543441344B34563469344D341F
:1000D0002034003420342034203445344C3445342A
:1000E0004B34543452344F344E3469344B3420340E
:0600F0002034203400342E
:100248008312080083120313DC000511803EBC29C9
:100258008312031305110130BC2102305B2983127C
:100268000313061301305B210617080083120313DA
:10027800061602305B21061202305B29F0000030BE
:10028800711870070310F00D0310F10CF108031931
:100298000800442983120313A0000A30F100200E3D
:1002A8000F394221F00020080F3970070800831227
:1002B8000313E2000430E3005330E400E40B622946
:1002C800E30B6029E20B5E2908008312031305156E
:1002D80075295D08EB005C08DC0A0319DD0A0620B5
:1002E800BC215D08EB005C080620003803190800F3
:1002F8006D2983120313DD0006123321DE01DE0AA5
:10030800DE0B84295D0888225C0888223321DE01FF
:10031800DE0ADE0B8D2906130800F401F50103102F
:10032800F30CF20C031C9F297008F40771080318DA
:10033800710AF5070310F00DF10D72087304031923
:100348000034932983120313DC00DD0106123321E4
:10035800DE01DE0ADE0BAE295C0888221622DD00EB
:100368003321DE01DE0ADE0BB72906135D0808001B
:1003780083120313DE005E0E0F39F0000608F03911
:1003880070048600851585115E080F39F00006088F
:10039800F03970048600851585110D30DF00DF0BFC
:1003A800D329080083120313A0000515200E0F3966
:1003B800F0000608F03970048600851585112008BC
:1003C8000F39F0000608F03970048600851585118C
:1003D8000D30A100A10BEE290800831203130511AB
:1003E8000F305B21033086008515851105305B21B0
:0803F800851585112130DC00A0
:10040000DC0B002A8515851105305B210230860042
:10041000851585110D30DC00DC0B0C2A2830BC2141
:100420000830BC210F30BC210630BC2983120313D5
:10043000DF01A03083168600831206120030861A70
:100440000130DF04E101E10AE10B242A3A21E00155
:10045000E00A0310DF0D0030861A0130DF04E101ED
:10046000E10AE10B312A3A21E00A08306002031C5C
:100470002A2AE0015F080139F0000730F10003107B
:10048000F00DF10B3F2A7008E0045F080239F0001C
:100490000530F1000310F00DF10B4A2A7008E0045A
:1004A0005F080439F0000310F00D0310F00D031085
:1004B000700DE0045F080839F0007007E0045F0881
:1004C0001039F0000310700CE0045F082039F000D0
:1004D0000310F00C0310F00C0310700CE0045F0824
:1004E0004039F0000530F1000310F00CF10B742AD4
:1004F0007008E0045F088039F0000730F100031055
:10050000F00CF10B7F2A7008E0046008DF0008009F
:1005100083120313DF0080308316860083120612D5
:100520005F0C031C952A8616962A8612E001E00AC3
:10053000E00B982A3A215F080239F0000310700C92
:10054000F000700C031CA62A8616A72A86128312B6
:100550000313E001E00AE00BAB2A3A215F080439FB
:10056000F0000310F00C0310700CF000700C031C72
:10057000BB2A8616BC2A861283120313E001E00A06
:10058000E00BC02A3A215F080839F0000310F00C94
:100590000310F00C0310700CF000700C031CD22A36
:1005A0008616D32A861283120313E001E00AE00BB9
:1005B000D72A3A215F081039F000F00E0F30F0050D
:1005C0007008700C031CE62A8616E72A861283122E
:1005D0000313E001E00AE00BEB2A3A215F0820391F
:1005E000F0000530F1000310F00CF10BF32A700855
:1005F000F000700C031CFE2A8616FF2A8612831256
:100600000313E001E00AE00B032B3A215F084039B5
:10061000F0000630F1000310F00CF10B0B2B70080A
:10062000F000700C031C162B8616172B86128312F3
:100630000313E001E00AE00B1B2B3A215F0880392D
:10064000F0000730F1000310F00CF10B232B7008C1
:10065000F000700C031C2E2B86162F2B8612831293
:100660000313E001E00AE00B332B3A298312E50083
:10067000E30103135C08E000E72C6408253A031D3E
:10068000DA2CFF30E100E201DF01A42CE5080319B8
:100690004D2B650884008313800163080800023035
:1006A000E0076002840083130008D82CDF0A5C2B6B
:1006B0000830E107FE30E1070230E0076002840005
:1006C00083130008E600840A0008E7005F18E71FAC
:1006D000702BE609E709E60A0319E70AE203712B22
:1006E000DF010B30E1076108F200F3016708F10058
:1006F0006608F000C9277008E4006108F200F30101
:100700006608F0006708F100C9277408E60075085C
:10071000E700E801E80AE90169086702031D922B76
:1007200068086602031CAF2B6108F200F301680839
:10073000F0006908F10091217408E8007508E900EB
:10074000E2038C2BE30AE5080319AD2B650884004E
:10075000831320308000E50AAF2B20302421E203F0
:100760006208803A7F3E0318A22B5F1CC42BE30A69
:10077000E5080319C22B6508840083132D3080001F
:10078000E50AC42B2D3024216108F200F30168082A
:10079000F0006908F100C9277408E8007508E9004D
:1007A00068040319F92B6908F3006808F200670868
:1007B000F1006608F000C9277408F0007508F10020
:1007C0006108F200F301C9277008E200803A763E22
:1007D000031CEC2B0730E207E30AE5080319F62BAC
:1007E0006508840083136208303EBF2B6208303EE8
:1007F000C32B0A306402031CFF2B0730E407E30A13
:10080000E5080319092C6508840083136408303E49
:10081000E22C6408303EE62CE30AE5080319172CA5
:1008200065088400831320308000E50A192C2030ED
:100830002421E2036208803A7E3E03180C2C023029
:10084000E0076002840083130008E400DA2C023021
:10085000E0076002840083130008E800840A0008AF
:10086000E900E40164086807EA006908EB006A0827
:100870000318EB0A062000380319402CE40A322C36
:10088000610864020318462C6408E1006108E21B59
:10089000722CFF3A6207031C722CE30AE508031965
:1008A000582C65088400831320308000E50A5A2CF8
:1008B00020302421E203462C69080313EB0068086A
:1008C0000620E400E80A0319E90AE30AE508031927
:1008D000702C65088400831364088000E50A722C7C
:1008E00064082421E103610F5C2CE72C5E08EB0017
:1008F0005D0806202A3A031D842C0230E0076002BE
:10090000840083130008A02C5E08EB005D0806201D
:10091000D03EE100DD0A0319DE0A5E08EB005D0847
:100920000620E40030306402031CA42C3A30640238
:100930000318A42C0A30F100610842216407D03E5C
:10094000E100DD0A0319DE0A5E08EB005D08DD0A3E
:100950000319DE0A0620E400003A0319462B2A3A5E
:1009600003194F2B043A0319762C763A0319582BA6
:100970003B3A03191A2C073A0319562B0B3A031961
:100980005A2B1C3A0319272C063A03195C2B0D3AF3
:100990000319582B30306402031CDA2C3A306402FD
:1009A0000318DA2C0A30F100620842216407D03EB5
:1009B000E200A42CE30AE5080319E52C650884008D
:1009C000831364088000E50AE72C640824215E088C
:1009D0000313EB005D08DD0A0319DE0A0620E400BC
:1009E000E408031D3D2BE5080319FA2C6508840073
:1009F0008313800163080800203083120313B600BC
:100A0000B700B800B900BA00BB00BC00BD00BE0012
:100A1000BF00C000C100C200C300C400C500C601C1
:100A2000C700C800C900CA00CB00CC00CD00CE0072
:100A3000CF00D000D100D200D300D400D500D60022
:100A4000D70103308316850080308600831285012C
:100A5000860107309F00FA305B21F1212C210C30F8
:100A6000BC21DC018E307D21A530DC0090307D2161
:100A70008130A621A8008039F0000730F100031072
:100A8000F00CF10B3F2D7008A000200B4C2DA8138B
:100A90002808DC0080307D21003026216A30DC000F
:100AA0000030DD006921403026215930DC00003063
:100AB000DD006921AC01FA305B21AC0A04302C0264
:100AC000031C5B2DAE0106123321BF30882281301A
:100AD000A621A8008330A621A4008530A621A60067
:100AE0008730A621A5008930A621A3008B30A6213E
:100AF000B5008D30A621A70033212C21260E0F39F9
:100B0000AD0026080F39B300240E0F39AA002408BF
:100B10000F39B100280E0F39A20028080F39A100A3
:100B2000250E0F39AB0025080F39B200230E0F39FF
:100B3000A90023080F39B000270E0F39AF0027088E
:100B40000F39B4003F30DD000030DE003308DA003A
:100B5000DB012D08D800D9015830DC0036303623AF
:100B60003F30DD000030DE003108DA00DB012A080A
:100B7000D800D9015830DC00393036232A30DD0066
:100B80000030DE002108DA00DB012208D800D9019C
:100B90005830DC003C303623003026213630DC0073
:100BA0008030DD0069210A302621350BDC2D2F3005
:100BB000DC000030DD0069213508023A031DE52D17
:100BC0001A30DC000030DD0069213508033A031DCE
:100BD000EE2D3530DC000030DD0069213508043AA7
:100BE000031DF72D5230DC000030DD00692135088F
:100BF000053A031D002E4B30DC000030DD0069217A
:100C00003508063A031D092E3A30DC000030DD00BD
:100C100069213508073A031D122E2130DC0000300F
:100C2000DD0069214530DD000030DE003208DA00E9
:100C3000DB012B08D800D9015830DC0047303623BF
:100C40004530DD000030DE003008DA00DB01290825
:100C5000D800D9015830DC004A3036232830DD0076
:100C60000030DE003408DA00DB012F08D800D9019B
:100C70005830DC004D303623403026214730DC0030
:100C80008030DD006921AC01FA305B21AC0A023012
:100C90002C02031C442E051C5A2EAE0A2E08073ABD
:100CA0000319AE01AC0196305B21AC0A02302C0274
:100CB000031C532EAE08031D612E003026210C307C
:100CC000BC212E0BA12E003026210E30BC21851C0C
:100CD000852EB30A33080A3A031D702EB301AD0AFC
:100CE0002D08023A031D7A2E3308043A031D7A2E8A
:100CF000AD01B30133080F39F0002D0EF039F03992
:100D00007004A600DC0084307D21861FA12EB30371
:100D1000AD08031D912E330F912E0230AD0003302C
:100D2000B300330F962E0930B300AD0333080F39EB
:100D3000F0002D0EF039F0397004A600DC0084308C
:100D40007D212E08023A031DE22E033026210E30AB
:100D5000BC21851CC62EB10A31080A3A031DB22EE9
:100D6000B101AA0A2A08063A031DBB2EB108031DC9
:100D7000BB2EAA01B10131080F39F0002A0EF0395B
:100D8000F0397004A400DC0082307D21861FE22E41
:100D9000B103AA08031DD22E310FD22E0530AA00AE
:100DA0000930B100310FD72E0930B100AA03310844
:100DB0000F39F0002A0EF039F0397004A400DC007D
:100DC00082307D212E08033A031D012F0A3026218F
:100DD0000E30BC21851CF72EB50A3508083A031DD4
:100DE000F32EB501B50A3508DC008A307D21861F57
:100DF000012FB50BFD2E0730B5003508DC008A3019
:100E00007D212E08043A031D452F403026210E3047
:100E1000BC21851C282FB20A32080A3A031D122F62
:100E2000B201AB0A2B08033A031D1D2F3208023A08
:100E3000031D1D2FAB01B201B20A32080F39F000B9
:100E40002B0EF039F0397004A500DC0086307D21CE
:100E5000861F452FB203AB08031D352FB208031DB3
:100E6000352F0330AB00B201B20A320F3A2F0930EE
:100E7000B200AB0332080F39F0002B0EF039F03915
:100E80007004A500DC0086307D212E08053A031D84
:100E9000872F433026210E30BC21851C6A2FB00AD3
:100EA00030080A3A031D562FB001A90A290B5F2FFB
:100EB0003008033A031D5F2FA901B001B00A3008C2
:100EC0000F39F000290EF039F0397004A300DC006E
:100ED00088307D21861F872FB003A908031D772F37
:100EE000B008031D772FA901A90A0230B000300F06
:100EF0007C2F0930B000A90330080F39F000290E0B
:100F0000F039F0397004A300DC0088307D212E0810
:100F1000063A031D632D483026210E30BC21851C66
:100F2000AD2FB40A34080A3A031D982FB401AF0A52
:100F30002F080A3A031DA22F34080A3A031DA22FD4
:100F4000AF01B40134080F39F0002F0EF039F03939
:100F50007004A700DC008C307D21861F632DB40354
:100F6000AF08031DB82F340FB82F0930AF00B400FD
:100F7000340FBD2F0930B400AF0334080F39F0002F
:100F80002F0EF039F0397004A700DC008C307D2181
:100F9000632DF601F401F50172087304031900349E
:100FA0001F30F6040310F60AF20DF30D031CD32FC5
:100FB000F30CF20C73087102031DE02F720870022B
:100FC000031CE82F7208F0027308031C730AF10275
:100FD000F40DF50DF60BF61AD82FF61FF42FF409C1
:100FE000F40A0319F503F5097408F2007508F30013
:100FF000761F0034F009F00A0319F103F1090034F7
:02400E0061FF50
:00000001FF
